:020000000C28CA
:10000800FE000308F1000408F2000A08F300C62BFA
:10001800F92B3A08D23EB0003B080318013EFB3EDC
:10002800B100B201B301A301A2010530A100A030C3
:10003800A0003308A7003208A6003108A500300840
:10004800A400F0212308B3002208B2002108B1005F
:100058002008B000A301A2010F30A100A030A00029
:100068003308A7003208A6003108A5003008A4000C
:100078002D212308B3002208B2002108B10020086E
:10008800B0003108BD003008BC000514AF010E30C7
:100098002F02031867283D08AE003C08AD002F0A60
:1000A80058280310AE0CAD0CFF3E031D55282D1C1F
:1000B800612883120313051564288312031305119D
:1000C800AF0A2D244B2805112D2405112D240511C7
:1000D8002D2405112D2405112D2405112D2405117C
:1000E8002D2405112D2405152D2405152D24051065
:1000F8000800A0000A30A100A2012008F900790D2B
:10010800790D0139F400740C83120313031C8E2833
:1001180006158F280611790EF400F40CD920031C5B
:100128009728861598288611790EF400D920031C83
:100138009F288614A0288610790ECC20790CF4000C
:10014800F40CD920031CAA280615AB280611790C33
:10015800F400D920031CB2288615B3288611790C1F
:100168000139F400740C83120313031CBD28861490
:10017800BE2886107908CC200130A1020030031C6B
:10018800A203A202210A0319220A03190800C0289F
:100198000139F400740C83120313031CD5280614C8
:1001A800D6280610061606120800740C0139F50048
:1001B800750C8312031308008312861280307D2089
:1001C80086163B08F5003A08F400752106307D20B4
:1001D8003E08F400F501752141087D2040087D2086
:1001E80020307D2046307D204D307D2020307D2000
:1001F8003B08F5003A08F40075214408303A031D1D
:1002080007292030C40044087D2043087D20420887
:100218007D202E307D2041087D2040087D204D30F6
:100228007D2048307D207A307D203630F400F5017D
:100238003A089C3EF6003B080318013EE63EF700EC
:1002480081227508B5007408B400340867230D20AE
:10025800232AA801A901AA01AB0123082204210429
:10026800200403196C29AC01AC0AA31B4129031013
:10027800A00DA10DA20DA30D38290310A80DA90DDD
:10028800AA0DAB0D23082702031D542922082602B4
:10029800031D542921082502031D5429200824027E
:1002A800031C66292008A4022108031C210FA502AB
:1002B8002208031C220FA6022308031C230FA702EF
:1002C80028140310A30CA20CA10CA00CAC0B412900
:1002D8002B08A3002A08A2002908A1002808A000CA
:1002E80008003030C000C100C200C300C40027307D
:1002F8007502103003197402031C9129C40AF030E6
:10030800F4070318F50AD830F5077B29C30A183013
:10031800F4070318F50AFC30F50703307502E830D6
:1003280003197402031C9C298A29C20A9C30B12132
:1003380000307502643003197402031CA729992937
:10034800C10AF630B121003075020A30031974026F
:100358000318A4297408C0070800F4070318F50A4D
:10036800FF30F5070800861277307D2086160030AA
:100378007D201F307D2011307D2011307D201F30E1
:100388007D2004307D200E307D2015307D20A40195
:10039800A40AA501053025020318DF29A50AA3012F
:1003A800083023020318DC29A30A24087D20D42955
:1003B8000310A40DCE297330A400A5010530250231
:1003C80003180800A50AF830A407861224087D201F
:1003D80086161F307D20E229F401F501F601F701A8
:1003E800201C0A2A2408F407250803110318013ED3
:1003F800031DF507260803110318013E031DF60720
:10040800270803110318013E031DF7070310A40D65
:10041800A50DA60DA70D0310A30CA20CA10CA00CF2
:100428002308220421042004031DF4297708A300CB
:100438007608A2007508A1007408A00008008316B9
:100448009C18232A9B0183123E08452203188B1708
:100458009C182C2A831203103E0D83169B008312CE
:100468003B08452203188B179C18382A031483125B
:100478003E0D83169B0083123A08452203188B17FA
:10048800080083169A0003108B1B03148B131C158A
:1004980055309D00AA309D009C141C110800533053
:1004A8008312A6000530A7000130A602031CA7038B
:1004B800260A0319270A031D582A861206118611CF
:1004C80086140610061606127430A6000130A7001E
:1004D8000130A6020030031CA703A702260A03194D
:1004E800270A031D6C2A2B307D2013307D200C3009
:1004F8007D2004307D20B7219C2BA001A101750827
:1005080074040319A62AA201A20AF51B8F2A031054
:10051800F40DF50D882A0310A00DA10D75087702BA
:10052800031D982A74087602031CA22A7408F6028E
:100538007508031CF703F70220140310F50CF40CDC
:10054800A20B8F2A2108F5002008F4000800822356
:1005580083123F08031908003F0BB32AFC228312B9
:100568003F08023A031DB92A212383123F08033AA0
:10057800031DBF2A17243F08043A031DC42A082470
:10058800FF30B6002F30B7000130B6020030031C30
:10059800B703B702360A0319370A03190800C82A2D
:1005A80003103E0D83169B001C141A088312BA0010
:1005B800BB01BB00BA0103143E0D83169B001C143B
:1005C8001A088312BA070318BB0A2A303B023130D3
:1005D80003193A020318F72A19303B026430031949
:1005E8003A02031808001030BA002730BB00080090
:1005F800FB308312BA070318BB0AFF30BB0722304F
:100608003B02603003193A020318152B1C303B02D9
:10061800853003193A02031C152B8430BA001C30AC
:10062800BB0019303B02643003193A020318202B2F
:100638003030BA002A30BB00E02805308312BA07F0
:100648000318BB0A1C303B02853003193A02031C0D
:10065800382B22303B02603003193A020318382B3A
:100668006030BA002230BB002A303B023130031917
:100678003A02031C432B6430BA001930BB00E0284F
:10068800F81083120313861BF814781183120313CE
:10069800061B7815781D522B0130532B0030F000C3
:1006A800F81D582B0130592B00307006031D78199E
:1006B800632BF818612B7816622B78127814F811CE
:1006C8007819F8150800A3008612C0307D20861618
:1006D800A5015030250203180800A40105302402A2
:1006E80003187F2BA50AA40A23082506031D722BCD
:1006F80024087D20722B2D307D206D2B8312BF01A5
:10070800CF3083168600831206188C2BBF01BF0AD0
:100718008618902B0230BF000619942B0330BF00B7
:100728008619982B0430BF00C03083168600080055
:10073800B530F600F701861201307D200130F6024F
:100748000030031CF703F702760A0319770A031D22
:10075800A22B861280307D2086160800FF30B80054
:10076800B9000130B8020030031CB903B902380AD5
:100778000319390A031DB52BE9235322D923E02095
:100788003224C42B01300B1C00398B1D0039003872
:100798000319CF2B44230B1073088A0072088400B6
:1007A80071088300FE0E7E0E090083169B011C143F
:1007B8001A088312BE0015303E020318E62BBE0845
:1007C800031DE82BBE01BE0AD42A8B0183168501BE
:1007D800C0308600073083129F008501860183168A
:1007E80081138B150B108B170800F801F901BA015A
:1007F800BB01BC01BD01BE01BF01C001C101C201F5
:10080800C301C4018301B22BBE0A15303E02031C8A
:100818000F2CBE01BE0AD422E0208312BF080319A0
:1008280008008223112CBE0B1B2C1430BE00D422CE
:10083800E0208312BF080319080082231D2C781CAE
:100848000800781E282CFC22781A2B2C21237810DB
:10085800E028000085150000851108002324AB2A34
:02400E00503F21
:104200000100FF0027004C002700A6002700E20065
:104210002800140028006E002800BE002800F000CE
:10422000290022002200560022007E002200A60063
:1042300023008C002600F70027004C002700A60072
:104240002700E2002800140028006E002800BE00AD
:104250002800F000FF00FF00FF00FF00FF00FF004C
:00000001FF
